:10F80000B240805A200132C23D409EF93140800210
:10F81000F24080005600F2400F005700C2435800EB
:10F82000C2432200F2403F002100F2403F00270087
:10F83000F24040002A00F24040002900C2432E005E
:10F84000B2401018B001B2400060B201B240C00036
:10F850004A00B240D2007201B24010026001B240D0
:10F860001000620182436401F2403F000002F24056
:10F870003F000102C2430202C24303024C4332D2A0
:10F880005A4220007AE03F007AF03F00C24A030269
:10F89000B240E070B201A2C2B001B2D00300B00128
:10F8A00092B3B201FD231A42B4010A110A110A11DE
:10F8B0007B407F004B8AC24B0102A2C3B001B24021
:10F8C000E060B201A2C2B001B2D00300B00192B3B5
:10F8D000B201FD231A42B4010A110A110A117B4038
:10F8E0007F004B8AC24B0002A2C3B001C293030245
:10F8F0001620F29043000002122CF2904300010205
:10F900000E2CF2903E0000020A28F2903E00010206
:10F9100006284C9307245C83B0122EF9033CB012E6
:10F920002EF96C4205433590F005FD2BA93F3D4073
:10F9300094F9054335909800FD3B3D409EF9054301
:10F9400035909800FD3B36400002774678423940BA
:10F950002E004757022C394017003D4094F90543CB
:10F9600035901700FD3B3D409EF905430599FE3B50
:10F970005883ED2336900402E8233D4094F9054373
:10F9800035901700FD3B3D409EF9F2C04000290034
:10F990003041004DF2E04000290015530013F2C041
:08F9A00040002900155300137B
:10FFE8000000000000000000000092F9000000007E
:08FFF80000000000000000F809
:00000001FF
